:020000040000FA
:06000000C0EF14F0120035
:06080000C0EF14F012002D
:06082A000100B0290000EE
:08083000B80000000800000000
:0808380004011151FE0A17E052
:10084000010A01E025D00001040EB16F0F0EE66E23
:10085000710EE66E0F0EE66EF4EC12F0E552E55204
:10086000E55271A002D07190AFD8689A11D0000102
:10087000040EB16F0401206B010E0001B66FB76B5F
:100880000001200EB26F040EB36F0001C19300D0BF
:100890001200D9CFE6FFE1CFD9FF050EE126020E07
:1008A0000001605D11E169516A116B116C110AE17F
:1008B0000DD904015B5105E1120E0001705D01E1EB
:1008C0008C8001D038D976D0030E605D11E169517A
:1008D0006A116B116C110BE104015B5107E1575177
:1008E000581159115A1102E0020E5B6FEFD862D015
:1008F00004010851800B5EE1000160515BE130C4EE
:1009000061F031C462F032C463F033C464F034C4C3
:1009100065F035C466F036C467F037C468F038C493
:1009200069F039C46AF03AC46BF03BC46CF03CC463
:100930006DF03DC46EF03EC46FF0DF6A04013E51BD
:10094000DF5C13E2DF50EA6A3F0FE96E040EEA2231
:10095000EF50E66EDF50EA6A700FE96E000EEA2291
:10096000E552E750EF6EDF2AE9D709C480F0CBD912
:10097000000918E0DED9000915E0F9D9800E000160
:100980006D5D03E1020E606F0CD06D510AE1040150
:10099000400E096F000E0A6F060E0B6F0001030E6A
:1009A000606F4CD8400E04010817087D880E0813AC
:1009B00065EC12F0050EE15C02E2E16AE552E16EDF
:1009C000E552E7CFD9FF1200F00E8C1695161E0ED9
:1009D000716E04011F0E096F300E0A6F040E0B6F4B
:1009E000880E086F0401000E0E6F060E0F6F400E8A
:1009F0000C6F1200D9CFE6FFE1CFD9FFE652AEEC83
:100A00000BF0F00E8C169516810EE66E000EE66E5B
:100A1000AEEC0AF0E552E552DF6EDF5007E08C8065
:100A20008C828C848C860001819102D000018181AE
:100A3000606BE552E552E7CFD9FF1200000170511B
:100A40001B0A3BE0340A36E02F0A31E01E0A2CE094
:100A5000040A27E0190A22E0290A1DE0020A19E027
:100A60000D0A15E0370A11E0C4D90001848184938E
:100A700084858497200E8E6F8F6B0401010E5B6F4F
:100A8000576B586B596B5A6B1BD083D919D0D3D97C
:100A900017D056DB15D082EC09F012D022EC0AF008
:100AA0000FD050EC0AF00CD05FEC0AF009D07CECCF
:100AB0000AF006D09EEC0AF003D0A6EC0AF000D0B3
:100AC0000001000E946F060E956F120004010CBF1A
:100AD000FDD74F0E0E6F040E0F6F0D0E0D6F400EF3
:100AE0000C170C7D880E0C1365EC12F004011F0E20
:100AF000096F300E0A6F040E0B6F0001606B12005D
:100B0000D9CFE6FFE1CFD9FF04010CBFFDD7FD0E21
:100B1000DBCF0EF4FE0EDBCF0FF4FC0EDBCF0DF4BB
:100B2000400E0C170C7D880E0C1365EC12F0E5528C
:100B3000E7CFD9FF1200D9CFE6FFE1CFD9FF050EED
:100B4000E12604015B5127E1400E575D000E585924
:100B5000000E5959000E5A591EE3400EE66E94C01D
:100B6000E6FF95C0E6FFCCDFE552E552E552400EC8
:100B70000001695F000E6A5B6B5B6C5B400E0401F9
:100B8000575F000E585B595B5A5B400E000194277B
:100B9000000E9523AED05B5101E185D0D880400E88
:100BA00000016955000E6A55000E6B55000E6C551C
:100BB00006E2400E106E116A126A136A08D069C00C
:100BC00010F06AC011F06BC012F06CC013F0010E8F
:100BD00010C0DBFF020E11C0DBFF030E12C0DBFFF3
:100BE000040E13C0DBFFDF6ADFCF10F0116A126A58
:100BF000136AD950010FE96EDACFEAFFEE50105CAC
:100C0000EE501158EE501258EE50135809E2DF50D2
:100C1000EA6A000FE96E060EEA22EF6ADF2AE4D7DD
:100C2000D880400E00016955000E6A55000E6B55C4
:100C3000000E6C5519E2400EE66E000EE66E060ED2
:100C4000E66E5EDFE552E552E552400E0001695F57
:100C5000000E6A5B6B5B6C5B400E0401575F000E1D
:100C6000585B595B5A5B1ED069C0E6FF000EE66E0A
:100C7000060EE66E45DFE552E552E5520001696B6E
:100C80006A6B6B6B6C6B69510401575F00016A51B1
:100C90000401585B00016B510401595B00016C5168
:100CA00004015A5B26D057C4E6FF94C0E6FF95C006
:100CB000E6FF26DFE552E552E552040157510001F7
:100CC000695F0401585100016A5B04015951000138
:100CD0006B5B04015A5100016C5B69C057F46AC038
:100CE00058F46BC059F46CC05AF4696B6A6B6B6B47
:100CF0006C6B050EE15C02E2E16AE552E16EE552E1
:100D0000E7CFD9FF12001F0E0001805D0CE1550EE8
:100D1000611908E1530E621905E1420E631902E1FF
:100D2000430E641903E0000E03D002D0010E00D080
:100D3000120000016E510F0817E36F51100814E301
:100D4000010E6F5D11E3800E6D5D02E0000E01D0BB
:100D5000010E106E6D5102E0000E01D0010E101058
:100D600003E0010E03D002D0000E00D0120065C0D7
:100D700053F466C054F467C055F468C056F40401D7
:100D8000550E4F6F530E506F420E516F530E526FF0
:100D90001200D9CFE6FFE1CFD9FF030EE126240EE2
:100DA000E66EE66A5C0E106E290E116E126A10C0B5
:100DB000E6FF11C0E6FF12C0E6FF000EE66E060E6B
:100DC000E66E73EC14F0136E070EE15E135004012F
:100DD000240E576F586B596B5A6B5B6B030EE15CBB
:100DE00003E200D0E16AE552E16EE552E7CFD9FFB8
:100DF0001200000182918293829582978289828B70
:100E0000828D829F836B8491849384958497849B45
:100E1000849D849F856B866B876B886B0A0E896FB8
:100E20008A6B8B6B8C6B8D6B8E6B8F6B906B916BFE
:100E3000926B936B1200D9CFE6FFE1CFD9FF280E5A
:100E4000E126010EDE6EDE6ADE6ADD6ADD52DD520B
:100E50000F0E00019B15106E240E10C0DBFF250E37
:100E6000DB6A260EDB6A270EDB6ADECFBCF0DECF44
:100E7000BDF0DECFBEF0DDCFBFF0DD52DD52240E7F
:100E8000DB5008E00001D890BC37BD37BE37BF3714
:100E9000E804F9E1030E00019C15106E100E10C05D
:100EA000DBFF110EDB6A120EDB6A130EDB6A140E17
:100EB0009DC0DBFF150EDB6A160EDB6A170EDB6AC0
:100EC000060E116EC00E9E1511C0E7FFE75204E03A
:100ED000E8427F0BE706FCE1106E180E10C0DBFF46
:100EE000190EDB6A1A0EDB6A1B0EDB6A100EDBCFF3
:100EF00014F0110EDBCF15F0120EDBCF16F0130E2F
:100F0000DBCF17F00A0E1F0B07E0D890143615360A
:100F100016361736E806F9E1140EDBCF18F0150E79
:100F2000DBCF19F0160EDBCF1AF0170EDBCF1BF05C
:100F3000020E1F0B07E0D890183619361A361B36EA
:100F4000E806F9E118501412195015121A50161229
:100F50001B501712D950180FE96EDACFEAFF145060
:100F6000EE10106E1550EE10116E1650EE10126E3F
:100F70001750EE10136E040E10C0DBFF050E11C0EB
:100F8000DBFF060E12C0DBFF070E13C0DBFF030EF4
:100F900000019F15106E1C0E10C0DBFF1D0EDB6ADA
:100FA0001E0EDB6A1F0EDB6A800EA015E844010BE3
:100FB000106E200E10C0DBFF210EDB6A220EDB6AF2
:100FC000230EDB6A1C0EDBCF14F01D0EDBCF15F0F9
:100FD0001E0EDBCF16F01F0EDBCF17F0010E1F0B1E
:100FE00007E0D8901436153616361736E806F9E1BC
:100FF000D950200FE96EDACFEAFF1450EE10106ED0
:101000001550EE10116E1650EE10126E1750EE10B5
:10101000136E080E10C0DBFF090E11C0DBFF0A0EB5
:1010200012C0DBFF0B0E13C0DBFFD9CFE9FFDACF15
:10103000EAFFEECF10F0EECF11F0EECF12F0EFCFCF
:1010400013F0020E146E156A166A176AD950080F4B
:10105000E96EDACFEAFFEE501426EE501522EE507C
:101060001622EE50172214501F0B07E0D8901036AE
:10107000113612361336E806F9E10C0E10C0DBFF0C
:101080000D0E11C0DBFF0E0E12C0DBFF0F0E13C0E2
:10109000DBFF010E106E116A126A136AD950040F39
:1010A000E96EDACFEAFFEE501026EE501122EE5034
:1010B0001222EE50132210C004F011C005F012C02D
:1010C00006F013C007F00C0EDBCF09F00D0EDBCFDE
:1010D0000AF00E0EDBCF0BF00F0EDBCF0CF0B0ECF6
:1010E00013F000C0B8F001C0B9F002C0BAF003C0FC
:1010F000BBF00001B807000EB95BBA5BBB5BBBC0BD
:1011000000F6BAC001F6B9C002F6B8C003F6BFC017
:1011100004F6BEC005F6BDC006F6BCC007F6040165
:10112000080E576F586B596B5A6B5B6B280EE15C5E
:1011300002E2E16AE552E16EE552E7CFD9FF120023
:10114000D9CFE6FFE1CFD9FF0E0EE126080E72C01F
:10115000DBFF070E73C0DBFF060E74C0DBFF050E5E
:1011600075C0DBFF040E77C0DBFF030E78C0DBFF2A
:10117000090E71C0DBFF04015B6B576B586B596B39
:101180005A6B030EDBCF10F0040EDBCF11F0126AA6
:10119000136AD950050FE96EDACFEAFFEE50102638
:1011A000EE501122EE501222EE5013221050000188
:1011B000B85D1150B9591250BA591350BB590CE2CD
:1011C0000401010E5B6F0001848184938485849700
:1011D000210E8E6F8F6B5ED0D950030FE96EDACF80
:1011E000EAFF000ED880EE54000EED5453E2030ED9
:1011F000DB06040E01E2DB06000EE66E060EE66E6E
:10120000D950050FE96EDACFEAFFEECFE6FFEECF59
:10121000E6FFEECFE6FFEFCFE6FF01EC0DF0106E3C
:10122000060EE15E1050E76E020EE7CFDBFFD950ED
:10123000050FE96EDACFEAFFEE2A000EEE22EE226B
:10124000EE22020EDB501EE104015B6B576B020EB7
:10125000586F596B5A6B0001000E946F060E956F14
:10126000D880000E04015755000E5855000E5955F0
:10127000000E5A5502E25FDCF3D7576B586B596B7F
:101280005A6BAAD70401010E5B6F576B586B596BF1
:101290005A6B00D00E0EE15C02E2E16AE552E16EAB
:1012A000E552E7CFD9FF1200400E04010817087D70
:1012B000880E081365EC12F0040108BFFDD709C4BD
:1012C00010F0116A126A136A10500001695F115020
:1012D0006A5B12506B5B13506C5B09C410F0116AAF
:1012E000126A136A10500401575F1150585B125074
:1012F000595B13505A5B0401400E096F0A27000E18
:101300000B231200D9CFE6FFE1CFD9FF100EE12663
:10131000040EDB6A0A0E72C0DBFF090E73C0DBFF2E
:10132000080E74C0DBFF070E75C0DBFF060E77C02A
:10133000DBFF050E78C0DBFF04015B6BD950050FA6
:10134000E96EDACFEAFF000ED880EE54000EED54BD
:101350006EE20401576B020E586F596B5A6BD880BE
:10136000000E04015755000E5855000E5955000E39
:101370005A5502E299DFF3D754EC0EF000090CE065
:1013800000018491848384958497270E8E6F8F6BE0
:101390000401010E5B6F1BD0000EE66E060EE66EBA
:1013A000D950070FE96EDACFEAFFEECFE6FFEECFB6
:1013B000E6FFEECFE6FFEFCFE6FFA4EC0DF0106EF8
:1013C000060EE15E1050E76E040EE7CFDBFF040E61
:1013D000DB5003E00401010E5B6FD950070FE96E8B
:1013E000DACFEAFFEE2A000EEE22EE22EE22050E02
:1013F000DB06060E01E2DB06D950050FE96EDACFF7
:10140000EAFF000ED880EE54000EED5408E204010D
:10141000400E096F000E0A6F060E0B6F07D0040115
:101420001F0E096F300E0A6F040E0B6F87D7100E58
:10143000E15C03E200D0E16AE552E16EE552E7CFFC
:10144000D9FF1200D9CFE6FFE1CFD9FFE652DF6A1C
:10145000DF50106E116A120E105C000E115813E26C
:10146000DF50EA6A820FE96E000EEA22EF50E66E64
:10147000DF50EA6A000FE96E060EEA22E552E750F5
:10148000EF6EDF2AE5D70401120E576F586B596BC8
:101490005A6B5B6B00D0E552E552E7CFD9FF1200E3
:1014A0000601030E006F016B026B036B04015B6BA3
:1014B000040E576F586B596B5A6B00D01200B3EC87
:1014C0000BF0F3CF10F0F4CF11F01050111007E033
:1014D00004015B6B576B586B596B5A6B0BD0000157
:1014E00084918483849584973A0E8E6F8F6B040168
:1014F000010E5B6F00D0120004015B6B7ADCB3EC71
:101500000BF0F3CF10F0F4CF11F0105011100EE1EA
:10151000000184918483848584973A0E8E6F8F6B4B
:101520000401010E5B6F0001819101D08C720401F6
:10153000576B586B596B5A6B00D0120004015B6BF0
:10154000576B586B596B5A6B00D0120004015B6BE0
:0C155000576B586B596B5A6B00D012009F
:04155C00D9CFE6FFFE
:10156000E1CFD9FF060EE126020EDB6A030EDB6A2D
:10157000FD0EDBCFE9FFFE0EDBCFEAFFEF6A8A86C6
:10158000E66A030EE66E020EE66EE8EC13F0E55234
:10159000E552E552640EE66E16DAE552DE6ADD6A61
:1015A000DECF10F0DDCF11F00A0E105C000E1158E6
:1015B00009E2E66896EC14F0E552DF2A010E01E339
:1015C000DB2AEED78A96010EE66EFDD9E552E66A71
:1015D000E66AE66AE66AE66AD1D8106E050EE15E52
:1015E0001050040EF3CFDBFF050EF4CFDBFF040E2B
:1015F000DB50FF0806E1010EF36E020EF3CFDBFFB6
:1016000093D0040EDB0405E0020EF36EF3CFDBFF94
:101610008BD0DE680F0EDD6EE66AE66AE66AE66A81
:10162000010EE66EABD8106E050EE15E1050040E92
:10163000F3CFDBFF050EF4CFDBFFDF06010E01E287
:10164000DB06040EDB5007E0D9CFE9FFDACFEAFF73
:10165000EE50ED10E1E1D9CFE9FFDACFEAFFEE502D
:10166000ED1007E1030EF36E020EF3CFDBFF5CD04B
:1016700016D026DBE76E030EE7CFDBFFDB500AE177
:10168000E66A030EE66EE66AE8EC13F0E552E55210
:10169000E55205D0040EF36E020EF3CFDBFFE66ACF
:1016A000020EE66EE66AE66A060EE66E67D8106E11
:1016B000050EE15E1050F8DA000907E0FD0EDBCF01
:1016C000E9FFFE0EDBCFEAFFEF82DE68DD6AD9CFED
:1016D000E9FFDACFEAFF000ED880EE54000EED5499
:1016E00014E2000EE66E060EE66EE66AE66AE66A4A
:1016F000E66A87D9106E060EE15E1050000905E01B
:10170000DF06010E01E2DB06E2D7D9CFE9FFDACF2F
:10171000EAFFEE50ED1005E1020EF36EF3CFDBFFB2
:1017200003D0020EDB5003D08A86DB5000D0106E4F
:10173000060EE15C02E2E16AE552E16E1050E5520C
:10174000E7CFD9FF12000A0EE66E3DD9E55281506F
:10175000100B100A01E0010E00D0120093888A8657
:1017600093969288120081A804D0F36AF46A05D097
:1017700004D0010EF36EF46A00D01200D9CFE6FF58
:10178000E1CFD9FF0B0EE126080EDE6EDD6A8A96E8
:10179000FE0EDB50040DF3CFF6FFF4CFF7FF340E4F
:1017A000F626280EF72208000A0EF5CFDBFFD950E7
:1017B000FA0FE96EFF0EDA20EA6E060EEECFDBFFBF
:1017C000070EEECFDBFF080EEECFDBFF090EEECFEC
:1017D000DBFFFE0EDB50040DF3CFF6FFF4CFF7FF77
:1017E000340EF626280EF722F62A000EF7220800FD
:1017F000050EF5CFDBFF0A0EDBCFE6FF96EC14F00B
:10180000E552090EDBCFE6FF96EC14F0E552080E28
:10181000DBCFE6FF96EC14F0E552070EDBCFE6FFD8
:1018200096EC14F0E552060EDBCFE6FF96EC14F0D2
:10183000E552050EDBCFE6FF96EC14F0E552FE0E06
:10184000DB50040DF3CFF6FFF4CFF7FF340EF6268E
:10185000280EF722020EF626000EF7220800F55099
:1018600013E0FE0EDB50040DF3CFF6FFF4CFF7FFCD
:10187000340EF626280EF722020EF626000EF72268
:101880000800F550010815E198D8E76E030EE7CF80
:10189000DBFFDF06010E01E2DB06030EDB50FF0873
:1018A00007E1D9CFE9FFDACFEAFFEE50ED10ECE126
:1018B0001ED0FE0EDB50040DF3CFF6FFF4CFF7FF82
:1018C000340EF626280EF722020EF626000EF72218
:1018D0000800F55002080BE170D86FD8E76E040ECF
:1018E000E7CFDBFF6AD8E76E030EE7CFDBFFFE0E24
:1018F000DB50040DF3CFF6FFF4CFF7FF340EF626DE
:10190000280EF722020EF626000EF7220800F550E8
:10191000010827E1030EDB6A020EDB6AFF0EF36E9D
:10192000020EDBCFF4FFF350F45C1BE2030EDB503E
:1019300018E1DE68DD6841D8E76E030EE7CFDBFF14
:10194000DF06010E01E2DB06030EDB5007E1D9CF13
:10195000E9FFDACFEAFFEE50ED10EDE1020EDB2AEF
:10196000DDD7E66896EC14F0E552FE0EDB50040D70
:10197000F3CFF6FFF4CFF7FF340EF626280EF7224A
:10198000030EF626000EF7220800F55001E18A86C4
:10199000030EDBCF10F0040EDBCF11F010C0F3FF0D
:1019A00011C0F4FF0B0EE15C03E200D0E16AE552E6
:1019B000E16EE552E7CFD9FF1200C968C7A0FED794
:1019C000C95000D01200D9CFE6FFE1CFD9FFB00E49
:1019D000CD6E9D80FD0ECF6E930ECE6E9E90CD800F
:1019E0009EA0FED7CD9000000000FE0EDB06FE0E8E
:1019F000DB500008EFE3CD909D90E552E7CFD9FF93
:101A00001200D9CFE6FFE1CFD9FF060EE126050E81
:101A1000DB6A95948384FB0EDBCF10F0FC0EDBCFEA
:101A200011F0FD0EDBCF12F0FE0EDBCF13F0090E2E
:101A30001F0B07E0D8901036113612361336E80621
:101A4000F9E110C0E6FF11C0E6FF12C0E6FF13C0C7
:101A5000E6FF070EE66E92DE146E050EE15E145090
:101A6000020EF3CFDBFF030EF4CFDBFF020EDB50E1
:101A700005E0050EF36EF3CFDBFF55D0DE68020EF6
:101A8000DD6E9BDFE76E040EE7CFDBFFDF06010EA6
:101A900001E2DB06040EDB50FF0807E1D9CFE9FFC6
:101AA000DACFEAFFEE50ED10ECE1D9CFE9FFDACF63
:101AB000EAFFEE50ED1004E0040EDB50FE0806E0F5
:101AC000060EF36E050EF3CFDBFF29D0DE6ADD6A6A
:101AD000DECF10F0DDCF11F0000E105C020E1158B9
:101AE00016E26BDFE66EF90EDBCF10F0FA0EDBCFFD
:101AF00011F0DE501024E96EDD501120EA6EE5523F
:101B0000E750EF6EDF2A010E01E3DB2AE1D7E6683A
:101B100096EC14F0E552E66896EC14F0E552E668AF
:101B200096EC14F0E5528A868394050EDB50106E15
:101B3000060EE15C03E200D0E16AE552E16E10506E
:101B4000E552E7CFD9FF1200D9CFE6FFE1CFD9FFA9
:101B5000060EE126050EDB6A95968386FB0EDBCF2B
:101B600010F0FC0EDBCF11F0FD0EDBCF12F0FE0EFD
:101B7000DBCF13F0090E1F0B07E0D890103611369B
:101B800012361336E806F9E110C0E6FF11C0E6FF91
:101B900012C0E6FF13C0E6FF090EE66EEFDD146E1D
:101BA000050EE15E1450030EF3CFDBFF040EF4CFFD
:101BB000DBFF030EDB5005E0050EF36EF3CFDBFF1A
:101BC00062D0FE0EE66E96EC14F0E552DE6ADD6A37
:101BD000DECF10F0DDCF11F0000E105C020E1158B8
:101BE00016E2F90EDBCF10F0FA0EDBCF11F0DE506B
:101BF0001024E96EDD501120EA6EEF50E66E96EC8F
:101C000014F0E552DF2A010E01E3DB2AE1D7E66892
:101C100096EC14F0E552E66896EC14F0E552CDDE51
:101C2000E76E020EE7CFDBFFDB500F0B050806E087
:101C3000080EF36E050EF3CFDBFF21D0DE6ADD6AFE
:101C4000BCDEE76E020EE7CFDBFFDF2A010E01E309
:101C5000DB2A020EDB5007E1D9CFE9FFDACFEAFF3A
:101C6000EE50ED10EDE1D9CFE9FFDACFEAFFEE500B
:101C7000ED1005E1060EF36E050EF3CFDBFFE6680F
:101C800096EC14F0E5528A868396050EDB50106EB2
:101C9000060EE15C03E200D0E16AE552E16E10500D
:101CA000E552E7CFD9FF120080A803D0010E03D080
:101CB00002D0000E00D01200D5EC14F08A8612007B
:101CC000D9CFE6FFE1CFD9FF130EE126020EDB6884
:101CD000F36E030EF3CFDBFF070EDB6A020EF36E2B
:101CE000080EF3CFDBFF090EDB6A0A0EDB6A0B0E70
:101CF000DB6A0C0EDB6A8A96080EDB50040DF3CF0C
:101D0000F6FFF4CFF7FF340EF626280EF722080070
:101D1000120EF5CFDBFFD950090FE96EDACFEAFFDB
:101D20000E0EEECFDBFF0F0EEECFDBFF100EEECF71
:101D3000DBFF110EEECFDBFF080EDB50040DF3CFFF
:101D4000F6FFF4CFF7FF340EF626280EF722F62A18
:101D5000000EF72208000D0EF5CFDBFF120EDBCFD1
:101D6000E6FF96EC14F0E552110EDBCFE6FF96ECA1
:101D700014F0E552100EDBCFE6FF96EC14F0E552BE
:101D80000F0EDBCFE6FF96EC14F0E5520E0EDBCF24
:101D9000E6FF96EC14F0E5520D0EDBCFE6FF96EC75
:101DA00014F0E5520ADEE76E040EE7CFDBFF020E09
:101DB000DB06030E01E2DB06040EDB50FF0808E140
:101DC000D950020FE96EDACFEAFFEE50ED10EAE1EA
:101DD000040EDB5006E0050EF36E070EF3CFDBFFBB
:101DE00049D0DE68020EDD6EE8DDE76E060EE7CF55
:101DF000DBFFDF06010E01E2DB06060EDB50FF080B
:101E000007E1D9CFE9FFDACFEAFFEE50ED10ECE1C0
:101E1000D9CFE9FFDACFEAFFEE50ED1004E0060E6D
:101E2000DB50FE0806E0060EF36E070EF3CFDBFF75
:101E30001DD0DE6ADD6ADECF10F0DDCF11F0100EAE
:101E4000105C000E115812E2B8DDE66EDECFE9FF3D
:101E5000DDCFEAFF960EE926000EEA22E552E750B2
:101E6000EF6EDF2A010E01E3DB2AE5D7E66896EC88
:101E700014F0E5528A86070EDB50106E130EE15CFB
:101E800003E200D0E16AE552E16E1050E552E7CF7F
:041E9000D9FF120064
:0C1E940004011051600BE842E842E842F3
:101EA000E842E842000901E055D01151070A51E02B
:101EB0000B0A4FE0070A40E0010A2CE00B0A28E079
:101EC000020A26E0030A22E0080A12E0010A0EE0F4
:101ED0000F0A0AE0030A01E03CD00001010EB16FD5
:101EE0000001040EC06F36D036D834D090D832D02E
:101EF0000001010EB16F0001C20EB26F000EB36F90
:101F00000001C1930001010EB66F24D0A8D822D0E1
:101F1000F6D820D00001010EB16F04011451000168
:101F2000B26FB36BC30EB227000EB3230001C1938F
:101F30000001010EB66F0ED00001010EB16F040159
:101F40001451EA6AC30FE96E000EEA2212C4EFFFD1
:101F500001D000D01200800E0401105D57E1135132
:101F6000030A34E0010A10E0030A01E04DD0000149
:101F7000010EB16F0001120EB26F260EB36F120E7A
:101F80000001B66FB76B40D00001010EB16F0401C4
:101F90001251F66EF76AD890F636F736B60EF62678
:101FA000260EF7220900F5CFB2F00A00F5CFB3F004
:101FB000020E0001F76AB225F66EB351F72209004E
:101FC000F5CFB6F00A00F5CFB7F01ED00001010E34
:101FD000B16F04011251F66EF76AD890F636F736F3
:101FE000BA0EF626260EF7220900F5CFB2F00A0047
:101FF000F5CFB3F0B2C0F6FFB3C0F7FF0800F5505D
:102000000001B66FB76B00D00001C1831200000160
:10201000010EB16F0F0EE66E710EE66E0F0EE66EDC
:10202000F4EC12F0E552E552E552010EE66EC30EF5
:10203000E66E000EE66EF4EC12F0E552E552E55263
:1020400012C4C2F00401125104E10001050EC06F78
:1020500005D00001060EC06FE4EC04F0120004018C
:10206000206B216B040110511F0B020A16E0030ABA
:1020700010E0010A01E035D00001010EB16F80A42B
:1020800002D0040120810001C1A102D004012083FB
:1020900028D00001010EB16F24D00001010EB16FF4
:1020A000040114510F0B080DF350116A000F106E4C
:1020B000040E11221451800B01E0010E040DF350A7
:1020C00000011024B46F000E1120B56FB4C0E9FFF9
:1020D000B5C0EAFFEF50040B03E00401010E206FCE
:1020E00000D00001B1050AE10001200EB26F040E1C
:1020F000B36F0001C1930001020EB66F120004011C
:10210000120510E110511F0B00090CE10001010E36
:10211000B16F030E0401115D03E10001C18102D022
:102120000001C191040112513AE110511F0B020844
:1021300036E114510F0B000932E00001010EB16FBE
:10214000040114510F0B080DF350116A000F106EAB
:10215000040E11221451800B01E0010E040DF35006
:1021600000011024B46F000E1120B56F030E04019E
:10217000115D07E1840EB4C0E9FFB5C0EAFFEF6E60
:102180000ED014AF06D0B4C0E9FFB5C0EAFFEF6AC5
:1021900006D0880EB4C0E9FFB5C0EAFFEF6E1200AA
:1021A0006C500BE1040100513C0BE842E8420D0881
:1021B00002E108D801D03CD804D0040E6C5C01E1E7
:1021C00047D81200D9CFE6FFE1CFD9FFE652000190
:1021D000B06BB16BB66BB76B4AEC0FF0DF6ADF50D8
:1021E000106E116A010E105C000E11581BE2000106
:1021F000B15101E017D0F76ADF34FE0BF736F66E07
:10220000C00EF626260EF7220900F5CF10F00800C2
:10221000F5CF11F004D011C0FAFF1050F96EFBDFBA
:10222000DF2ADDD7DDD8E552E552E7CFD9FF12002E
:10223000020E0001B05D0AE196D8040100BD03D092
:10224000C80E006F02D0880E006F01D00FD91200A7
:10225000040E0001C05D0AE112C46EFF6E5000085A
:1022600003E2050EC06F02D0030EC06F0001B0057F
:102270000AE10BD8040104BD03D0C80E046F02D0DC
:10228000880E046F01D0F2D81200D9CFE6FFE1CF5B
:10229000D9FF020EE1260001100EB65D000EB759FF
:1022A00005E2B6C0DEFFB7C0DDFF03D0100EDE6E64
:1022B000DD6A040104930491010EDB500413DFCFA7
:1022C00005F4000EDB500001B65F010EDB50B75B7A
:1022D000200EB46F040EB56F0001C1A31ED0D9CF7C
:1022E000E9FFDACFEAFFEE50ED1016E0B2C0F6FFDC
:1022F000B3C0F7FF0800F550B4C0E9FFB5C0EAFF6E
:10230000EF6E0001B42B000EB523B22BB323DF0612
:10231000010E01E2DB06E3D71CD0D9CFE9FFDACF0B
:10232000EAFFEE50ED1015E0B2C0E9FFB3C0EAFFDE
:10233000EF50B4C0E9FFB5C0EAFFEF6E0001B42B67
:10234000000EB523B22BB323DF06010E01E2DB063C
:10235000E4D7020EE15C02E2E16AE552E16EE55289
:10236000E7CFD9FF1200D9CFE6FFE1CFD9FF020EA8
:10237000E126030E04010015E76E010EE7CFDBFF37
:1023800001C4DFFFDE500001B627DD50B723200E69
:10239000B26F040EB36FD9CFE9FFDACFEAFFEE5088
:1023A000ED1014E0B2C0E9FFB3C0EAFFEF50B4C0D3
:1023B000E9FFB5C0EAFFEF6EB42B000EB523B22BD8
:1023C000B323DF06010E01E2DB06E5D7020EE15C76
:1023D00002E2E16AE552E16EE552E7CFD9FF120071
:1023E0006D980001B1510CE10401100E016F100E47
:1023F000026F040E036F840E006F0401046F35D06A
:10240000040110AF22D00001B6510401165D000195
:10241000B7510401175904E216C4B6F017C4B7F057
:1024200034DF0001010EB06F0401100E016F100EB9
:10243000026F040E036F800E006F0401200E066F02
:10244000040E076FC80E046F10D00001020EB06FAB
:102450000401056BC80E046F0401100E016F200EFD
:10246000026F040E036FC80E006F12000001B06B04
:102470000401100E016F100E026F040E036F880E20
:08248000006F0401046B12005F
:0824880080A203D06DA60FD85D
:1024900002D06DB613D80001C00508E16DBA06D0B0
:1024A000686A696A69806988020EC06F12006D6A85
:1024B000696A6D860001010EC06F12006D6A696A5B
:1024C0000001C06B12005EEF12F00001C05101E18B
:1024D0003AD06850040B04E06950040B01E041D885
:1024E0006DB231D06850010B04E06950010B01E07E
:1024F00059D86850100B04E06950100B01E024D843
:102500006850400B04E06950400B01E040D868502F
:10251000200B04E06950200B01E03BD86850020B0F
:1025200004E06950020B01E03BD8030E0001C05DDE
:1025300001E209D06850080B06E06950080B03E07F
:10254000D0EC10F068961200698468986D82A19AA8
:10255000F290A08AF2860300F2B007D8A09AF29611
:1025600012006D926994689412000001C1A10ED00E
:10257000F8DF6D840001080EC46F070EC56FC40735
:10258000000EC55BC451C511FAE16D941200689C40
:10259000120070A003D036EC12F07090689A12000E
:1025A000689212006A6A686A9F0E6B6E7B0E696E93
:1025B0006E6A0F0EE66E710EE66E0F0EE66E14D8A2
:1025C000E552E552E552160E706E68A602D0689686
:1025D000FCD76D9836EC12F00001C1910001C26B7E
:1025E0000001030EC06F1200D9CFE6FFE1CFD9FF83
:1025F000FD0EDBCFE9FFFE0EDBCFEAFFFC0EDB506A
:1026000004E0EE6AFC0EDB06F9D7E552E7CFD9FF0E
:022610001200B6
:0E2612001201000200000010D80409000100AF
:102620000102000109022000010100C0320904007A
:10263000000208065000070581024000000705015E
:10264000024000000403090434034D0069006300E4
:1026500072006F0063006800690070002000540081
:102660006500630068006E006F006C006F0067001B
:102670007900200049006E0063002E003A034D00EF
:102680006900630072006F006300680069007000F9
:1026900020004D006100730073002000530074009F
:1026A0006F00720061006700650020004400720046
:1026B00069007600650024262426442648267C26C8
:0226C0003808D8
:0E26C2002A0EF66E080EF76E000EF86E00017E
:1026D0000900F550AB6F0900F550AC6F03E1AB6733
:1026E00001D03DD00900F550A66F0900F550A76F45
:1026F0000900F550A86F09000900F550E96E0900BE
:10270000F550EA6E090009000900F550A96F0900AB
:10271000F550AA6F09000900F6CFADF0F7CFAEF083
:10272000F8CFAFF0A6C0F6FFA7C0F7FFA8C0F8FF2C
:102730000001A95302E1AA5307E00900F550EE6E2B
:10274000A907F8E2AA07F9D7ADC0F6FFAEC0F7FFB8
:10275000AFC0F8FF0001AB07000EAC5BBFD71200A3
:1027600004500902F3CF00F0F4CF01F00A02F35055
:102770000126000EF420026E04500B02F3500226D4
:10278000000EF420036E04500C02F3500326055093
:102790000902F3500126F4500222000E03220550D4
:1027A0000A02F3500226F450032205500B02F350A4
:1027B000032606500902F3500226F4500322065065
:1027C0000A02F350032607500902F35003261200B1
:1027D000D9CFE6FFDACFE6FFE1CFD9FFE2CFDAFFCC
:1027E0003F0EC716C66AFD0EDB50C612FB0EDB504D
:1027F000C712FC0EDB50030A09E0010A04E0020ADA
:1028000006E1C78C04D0C78CC68801D0C688FD0EEF
:10281000DB50050A03E0010A03E1928A938201D0AA
:1028200093929380949EC68AE552E5CFDAFFE7CF74
:04283000D9FF1200BA
:0C2834004095000041F9000049AF000190
:102840004A1B00014CC300004DAF020050FF0000C6
:1028500051FF000152FF000158FF000159FF000124
:1028600060FF000061FF000062FF000063FF0000E6
:1028700064FF000065FF000066DF01007189010050
:1028800069E50000777300007A2503007B250000CE
:1028900005D822D849EC04F0FCD712000F0EC11263
:1028A00092829284140E6F6E0001C06B0001C16BA6
:1028B0000001C26B938881A80DD00001C66BC76B65
:1028C000880EC65D130EC75904E2C62B000EC7233F
:1028D000F7D7F1D7FAEF04F044EC12F06FBE02D054
:0628E00065EC12F012008D
:0A28E600FB0EE3CFF6FFFC0EE3CF7C
:1028F000F7FFFD0EE3CFF8FFFE0EE3CFE9FFFF0E7B
:10290000E3CFEAFFE9CFF3FFEACFF4FFF90EE3509C
:1029100003E1FA0EE35009E0F90EE30602E2FA0ED3
:0C292000E3060900F5CFEEFFF1D712002E
:04292C00D9CFE6FF1A
:10293000DACFE6FFE1CFD9FFE2CFDAFFFD0EDB50C1
:10294000C96EC6AE02D0FF0E03D0C7A0FED7000EE0
:0C295000E552E5CFDAFFE7CFD9FF120017
:04295C0000800402F1
:10296000200000004D6963726F6368704D6173737E
:102970002053746F72616765202020203030303121
:1029800013EE00F023EE00F0F86A0F9C61EC13F0F8
:0C299000D7EC14F048EC14F0FBD7120058
:04299C0000EE00F059
:0A29A0000F0EEE6AEA62FDD7120086
:0429AA00C69A1200B7
:0229AE00120015
:0829B00000000000000000001F
:00000001FF
